:0300000002007A81
:200008000000E2FBEAF2802C0000E0FBEAF08024E6B50202EBF62200E2B50202EBF22200DE
:20002800E0B50202EBF02230F6E0A88220F5D3EAC6F582228B822230F6E6A88220F5D980EE
:01004800CFE8
:0E00D300E4F514F515F516F517F518020049B9
:0300490002028828
:2000E100759850758920758DFD758BFDC2ACC2AFD28ED299C29822AF8210990280FB8F99E3
:20010100223098FD859982C29822AF82BF0A0A75820DC0071200F8D0078F820200F812010D
:2001210002AF82BF0D027F0A8F82C00712010BD0078F8222AD82AE83AFF08D828E838FF096
:20014100120876FC60188C820DBD00010EC007C006C00512010BD005D006D00780DC22AD96
:2001610082AE83AFF08D0B8E0C8F0DA809A90AC007C006C005C001C00012011FAC82D000F7
:20018100D001D005D006D0078C08BC0D028022740AB50802801B18B8FF0119E84960128D19
:2001A100828E838FF0E508120826A3AD82AE8380BE8D828E838FF0E4120826C00BC00CC0A4
:2001C1000D8D828E838FF012004C1581158115816002800790000075F00022850B82850CAF
:2001E10083850DF022AE82AF83752D96752E08752F8090000E75F040C007C0061207E6D0CF
:2002010006D007C3EE9410EF9427400FEE24F0FEEF34D8FFE50E04F50E80E8C3EE94E8EF3A
:200221009403400FEE2418FEEF34FCFFE50F04F50F80E8C3EE9464EF9400400FEE249CFE06
:20024100EF34FFFFE51004F51080E8BE0A00400BEE24F6FEE51104F51180F0EE2512F51261
:2002610090000E75F040020135AE82AF831EBEFF011FEE4F6010758220C007C00612010B36
:20028100D006D00780E7221200E175820A12010B90002212026A90089C75F08012013590F4
:2002A100000F12026A9008A275F0801201357F00EF75F020A42426FD740E35F0FE8D028EA9
:2002C100037C007509208C0A8A828B838CF0C007C006C005120160D005D006D0078D828EF0
:2002E10083E0FDBD440280030F80C51F751900751A008F057E001DBDFF011EAB1A7C00C379
:20030100ED9BEE64808CF063F08095F04051E51A75F020A42426FD740E35F0FE7C008D827E
:200321008E838CF0C00712085EAD82AE83D007AB197C00C3EB9DEC9E5021E51A75F020A40B
:200341002426FD740E35F0FE7C008D828E838CF0C00712085EAD82D0078D19051A8093EF8C
:20036100C313FE7419C39EF51C2FF51DE519C313FE7423C39EF5202519F521751A00751B16
:2003810000E51A75F020A42426FD740E35F0FE7C008D828E838CF0C00712085EAD82AE8391
:2003A100D007AB1B7C00C3EB9DEC9E505DE51A75F020A42426FD740E35F0FEE51B2DF582E9
:2003C100E43EF583E0FEBE2A3CAD1C7E00AB1A7C00EB2DF52DEC3EF52E900047C0071208B9
:2003E10041AD82AE83D007ED2401FDEE3400FEE51B25202DF582E43EF5837401F00516E46E
:20040100B516020517051B020382051AC3EF951A400302037F9008E375F080120135751FC8
:2004210002751E30752302752244751A01AE1C7F001EBEFF011FAC1A7D00C3EE9CEF64804A
:200441008DF063F08095F0400A75820A12010B051A80DA75820A12010BE51C75F047A42450
:2004610001FE740035F0FF8E248F25752600851C1AC3E51D951A5003020540AE207F008E3F
:20048100828F8312026AE5202524F527E43525F52885262985201BC3E521951B500302051D
:2004A1002AAD27AE28AF298D828E838FF01208766013AD27AE28AF298D828E838FF01208B2
:2004C10076FDBD0318AD27AE28AF298D828E838FF0E412082675822012010B803FAD27AE15
:2004E10028AF298D828E838FF0740112082675822A12010BC3E51A951E5003851A1EC3E53B
:200501001F951A5003851A1FC3E51B95225003851B22C3E523951B5003851B23051B05278F
:20052100E4B52702052802049875820A12010B051A74472524F524E43525F525020472E51D
:200541001D04F51AE51A24CE400A75820A12010B051A80F09008E675F080120135851482BB
:200561008515831201E69008F375F0801201358516828517831201E6E518601490090275F6
:20058100F080120135AE187F008E828F831201E6E516451770012212011F851E1C851F1DA6
:2005A1008522208523210514E4B514020515E4F516F517F51874FE251C4006751C027518A7
:2005C10001E51D24CF500A751D30AF1874022FF51874FE2520400A752002AF1874042FF594
:2005E10018E52124BB500A752144AF1874082FF518AE1C7F00EE24FFF52DEF34FFF52E90F9
:200601000047120841AE82AF83EE2401FEEF3400FF8E248F25752600E51C14F51AAE1D7F33
:20062100000EBE00010FAC1A7D00C3EE9CEF64808DF063F08095F050030207DBE520252420
:20064100FDE43525FEAF26ED24FFF527EE34FFF5288F29E52014F51BAE217F000EBE000125
:200661000FAC1B7D00C3EE9CEF64808DF063F08095F050030207CB7F00E52724B8F52AE59F
:200681002834FFF52B85292CAC2AAD2BAE2C8C828D838EF012087630E0027F01052AE4B5F6
:2006A1002A02052BAC2AAD2BAE2C8C828D838EF012087630E0010F052AE4B52A02052BAC39
:2006C1002AAD2BAE2C8C828D838EF012087630E0010F7447252AF52AE4352BF52BAC2AADE1
:2006E1002BAE2C8C828D838EF012087630E0010F152A74FFB52A02152B152A74FFB52A0242
:20070100152BAC2AAD2BAE2C8C828D838EF012087630E0010F7447252AF52AE4352BF52B37
:20072100AC2AAD2BAE2C8C828D838EF012087630E0010F052AE4B52A02052BAC2AAD2BAE64
:200741002C8C828D838EF012087630E0010F052AE4B52A02052BAC2AAD2BAE2C8C828D8356
:200761008EF012087630E0010FAC27AD28AE298C828D838EF01208766027BF02004005EF23
:2007810024FC5013AC27AD28AE298C828D838EF0740312082680260516E4B51620051780D7
:2007A1001CBF0319AD27AE28AF298D828E838FF074021208260516E4B516020517051B055D
:2007C10027E4B527020528020659051A74472524F524E43525F52502061E151C1520051D5F
:0507E100052102041FC8
:200896003030303030004C4946450A00435245415449564520434F4D505554494E47204D92
:2008B6004F52524953544F574E2C204E4557204A45525345590A0A0A454E54455220594FBF
:2008D6005552205041545445524E3A0A000A0A0047454E45524154494F4E3A20000909501D
:1608F6004F50554C4154494F4E3A200020494E56414C4944200090
:2007E60085823085833185F032AA2DAB2EAC2FA830A931AF328A828B838CF0120876FEA3F7
:20080600AA82AB83888289838FF0EE120826A3A882A983EE70DF8530828531838532F02246
:0600A900E478FFF6D8FD2B
:200087007900E94400601B7A0090090C782675A012E493F2A308B8000205A0D9F4DAF275D3
:0200A700A0FFB8
:1B08260020F71130F6138883A88220F509F6A8837583002280FEF280F5F022D1
:1D084100E582852DF0A4C582C0F0852EF0A4D0F025F0C583852DF0A42583F583220A
:2000AF007800E84400600A790175A000E4F309D8FC7825E84412600C7913900001E4F0A305
:0400CF00D8FCD9FA86
:18085E00AA82AB831208766003A380F8C3E5829AF582E5839BF5832242
:20004C00E58124FCC3C8C0E0E608467006E58245836016C08218E58296F58208E58396427E
:1B006C008208E5F0964582D082C8D0E0C822758132120892E582600302004920
:1C08760020F71430F6148883A88220F507E6A88375830022E280F7E49322E02291
:040892007582002249
:00000001FF
